:100000000C94F0250C94BF22189518951895189506
:10001000189518950C946D221895189518951895A3
:10002000189518950C9444221895189518951895BC
:100030001895189518951895189518951895189558
:100040001895189518951895189518951895189548
:1000500018951895189518950000000103070F1FB3
:10006000040E1F1F1F1F1F1F00000010181C1E1F43
:100070001F0F0703010000001F1F1F1F1F1F0E047B
:100080001F1E1C1810000000080C0E0F0E0C08009C
:1000900002060E1E0E0602004C462D534D414C4CDE
:1000A00020204C462D4D454449554D204C462D4C65
:1000B0004152474520204C46322D534D414C4C2057
:1000C0004C46322D4D454449554D4C46322D4C4100
:1000D0005247452050422D4D454449554D205072C0
:1000E0006F436F6E6475637450726F4D61736B2DE7
:1000F000504450726F4D61736B2D50434652342003
:10010000312E356D6D2046523420312E356D6D20E7
:1001100046523420312E356D6D2046523420312E1A
:10012000306D6D2046523420312E306D6D20465298
:100130003420312E306D6D2046523420312E356DF5
:100140006D2046523420312E356D6D20507265641D
:10015000727920202020506F73746375726520209F
:10016000AAAAAAA0A0A096A050A096A0AA96A0AACB
:10017000A01E0A1EFAFF04FA040EE6A050A04B557A
:100180005F3C46505A000000505A64505A645A036B
:100190000306383A3A3A3A3A3A858A8A0000100019
:1001A000101000000000E6E6E6E6E6E6C8A050A073
:1001B0006464646464645A1E00000D0D0D0D0D0D21
:1001C0000D0D0D0DE6E6E6E6E6E6C8A050A0646477
:1001D000646464645A1E00000C0C0C0C0C0C0C0CB7
:1001E0000C0C00C8455343454E5456455253494F95
:1001F0004E2020332E31314E4F2050524F46494C25
:1002000045205245434F524445522153454C4543A6
:1002100054204F50454E2F434C4F534550524F465C
:10022000494C4520202053455454494E47532020E3
:1002300053544152542050524F4645444954205043
:10024000524F4620504342204C4546542052494785
:10025000485443454E5452554E4E494E474E4558CC
:10026000542050484153452B35205345434F4E446D
:10027000532B35204D494E5554455343414E43452C
:100280004C20414C4C5343524F4C4C26454E5453FA
:10029000484F5254204E414D4545585452412049F3
:1002A0004E464F5741524D555020505245484541BA
:1002B00054505245482054454D50205052454820F6
:1002C00054494D45205245464C4F57205245464CC7
:1002D0002054454D50205245464C2054494D452010
:1002E0005245464C205057522020434F4F4C4457C4
:1002F0004E434F4F4C205350454544434F4F4C20A5
:1003000054494D45205345432F4D494E20202053FD
:1003100045434F4E44532020204D494E555445539C
:100320002020204D554C5449205A4F4E454F4E4C9D
:1003300059205245464C205354455031265245468B
:100340004C5331265332265245464C535445503176
:10035000205057522053544550312054454D50534E
:10036000544550312054494D455354455032205046
:1003700057522053544550322054454D5053544504
:1003800050322054494D4553544550312020535448
:1003900045503220203130302520504F57455237BC
:1003A000352520504F5745522035302520504F5786
:1003B00045522043454E544552203530254C434448
:1003C000205649455720204C4344203343482020A1
:1003D000204C4344203743482020204C43442031C4
:1003E00043482020204C43442035434820202020EF
:1003F000202020B043454C202020202020B0434521
:100400004C20202020202020534543202020202045
:1004100020204D494E202020202020202025202053
:1004200020464143544F52592050524E6F204F4660
:100430002050524F4631302050524F4627532032E1
:10044000302050524F4627532033302050524F46D1
:100450002753204E322053455454494E474E3220A4
:100460004F4E20202020204E32204F464620202074
:10047000204E3220434845434B2020202020206C32
:100480002F682020204C4F4144494E47204641438D
:10049000544F5259204441544120202020202020F4
:1004A0002020444F4E45202020494E534552542091
:1004B00052454D4F564520505245535320454E54BA
:1004C000265741524E494E4721204F50454E494EE6
:1004D0004720434C4F53494E47445241574552459C
:1004E00052524F522121212020445241574552203F
:1004F000424C4F434B4544212020204E3220464C55
:100500004F5720544F4F204C4F5721204E322046FA
:100510004C4F5720544F4F204849474821434845A6
:10052000434B204D414E55414C412020204220203C
:1005300020432020204420202020C309D109E109A4
:10054000FD09F1090B0A1B0A270A850A8A0AA00A73
:10055000A00AA00AA00AA00AA00AA00AA00AA00A4B
:10056000A00AA00AA00AA00AA00A390A480A570A43
:10057000650A700A7B0A03E006B900E007B9379AFA
:1005800008950AB700640ABF05B7026005BF0BB73C
:1005900000640BBF0895979802E3A4D00CE01BD031
:1005A0001ED01DD09FD008E016D09CD018E211D0EC
:1005B0000DD01CE00ED00AD00BD004E193D016E091
:1005C00008D00AE08FD002E38DD0089502E08AC0FF
:1005D00011E000E053C005BB06D00AE0089582D0C8
:1005E00002D00AE00895AE9AAE98089538E001303E
:1005F00009F43CE0113009F43260213009F4316033
:10060000132FE7DF0895E4DF04E16CD00895202F75
:100610002A95123011F4022F0054113011F4022FD8
:100620000058133011F4022F0C56143011F42C52D0
:10063000022F102FCEDF0895BA93AA938A93D80180
:10064000822F04C01D9101E019D08A958823D1F72B
:100650008991A991B9910895AA939A938A93C8010F
:10066000A22F06C0FC011591CF0101E007D0AA9589
:10067000AA23C1F789919991A99108958A93812F0D
:10068000013011F4AF9A01C0AF9887FB16F4AA9A13
:1006900001C0AA9886FB16F4AB9A01C0AB9885FB03
:1006A00016F4AC9A01C0AC9884FB16F4AD9A01C064
:1006B000AD9899DF83FB16F4AA9A01C0AA9882FB31
:1006C00016F4AB9A01C0AB9881FB16F4AC9A01C04A
:1006D000AC9880FB16F4AD9A01C0AD9884DF76DF4C
:1006E00089910895392F482F10E007C00000019626
:1006F000803426E09207D4F31395101718F480E0A5
:1007000090E0F6CF842F932F089510E462DF20E469
:1007100008E510E0A1DF08950CE50DB9689A0EB167
:100720000FB1089500E00FBD05E00EBD04E008BF65
:1007300006EF0CBD02EC0DBD02E005BD00E408BFF4
:1007400005E004BD089510E010BD09B906E800BD3C
:1007500008E10AB9089504D0E2D201E097D70895DC
:1007600001E00ABB0FEF0BBB00EB07BB0FE008BBC0
:100770000FEF04BB00E005BB08EF01BB0CE702BBB9
:1007800000E000934F010E94CB0244D02DE00AEE1E
:1007900011E00E942C030E9492030E94BB0200E021
:1007A0000FB90E948C030E94C10200E00E94A303C3
:1007B00000E202B90FEF03B906B7046006BF0E945A
:1007C000432400915701002389F414E02ED024E142
:1007D00007EF11E00E942C0321D004C00AEF0E9411
:1007E000720312D00091FA000630C0F321D00895B0
:1007F0000091FA0010E0E00FF11F24910091FA003F
:10080000F801EA5EFE4F2083EAEFF0E000810395F5
:100810000083089512E004E00C94070300E00093C5
:10082000FA0008950E94030311E001E00C9407030D
:1008300001E010E0EAE5F1E00083118308958A9376
:10084000F3DF5FD003C0182F92D083958330D8F3A5
:1008500054D02091BE0030E004E066D212E005E002
:100860000E94070316E083D012E038D017E07FD053
:1008700013E0DBDF23E004EE11E056D002E10E943A
:10088000070323E007EE11E00E942C0342D080E032
:1008900004C0182F1D5F6BD083958330D0F362D0D6
:1008A0000E94EF1F13E017D00E9400200091FF006C
:1008B000013049F421E00BD012E00091FC000A5F06
:1008C0000E94070302C020E002D08991089510E041
:1008D00001E00C94F60206E00C94070300E10C948E
:1008E0000703008174D22091BE0030E001E210E0E5
:1008F000039F029F002D110D089511E003E10C9458
:1009000007030E94DD1F11E00AE00E94070380E058
:10091000089514E00AE00C94070311E007E00E9438
:10092000070328E001EC14E00E942C0313E0089573
:100930000E942C0314E005E00E9407032CE00DE167
:1009400015E008950E942C0324E002EA14E00E94BE
:100950002C0313E002E10E94070323E007EE11E0FD
:100960000E942C0312E006E00C940703108101E0C2
:100970000C943E030E943E0321E001EB10E00E9434
:100980001C0320E030E002E00E94CE221FED01E0D7
:100990000E943E0321E00FEA10E00C941C03E1D01A
:1009A0008A9342DFAEDF03C0182FE1DF83958330E7
:1009B000D8F3D1D06CF0E0D024E000EA10E00E943F
:1009C0001C039BDFEAE5F1E0B5D004E0ADD10EC039
:1009D0000091F700013051F400E00E945B1FCCD081
:1009E000AED023E005EA10E00E941C0313DF9ED086
:1009F00021E019F409EA10E002C00BEA10E00E94BD
:100A00001C03B0DF2AE00FEB10E00E941C0312E091
:100A100001E10E94070385D07CD074D00091FC00D6
:100A2000043621E019F40DEA10E002C00FEA10E0EC
:100A30000E941C0312E0F9DE79D011F460D001C0ED
:100A400059D07FD00091F500002329F48DD099DF93
:100A500097D00E942C030091F5000130B9F484D0A6
:100A600090DF8ED061DFE1DE21E08CDF14E0DDDE9F
:100A700025E008E412E058DF31DF22E083DF14E0F4
:100A80002DDF25E00DE412E00E942C030091F5001B
:100A9000023041F414E001E0A2D092D082D078D0AC
:100AA00001E068DF0091F5000330E1F414E001E0BB
:100AB00096D086D076D06CD001E05CDF13E0B5DE56
:100AC00021E003EB10E00E941C0321E051D013E071
:100AD00001E10E94070321E005EB10E00E941C03E6
:100AE00022E046D001D008958991A991B991089545
:100AF00000811181E9E2F1E0089500811181E7E2CE
:100B0000F1E00895980103E00FC1E3EDF0E000810A
:100B1000118142E050E00C945E26E4E4F1E024818F
:100B20003581E0E0F1E00081118108950091F40049
:100B30000023089520813181215030400895EDE453
:100B4000F1E02081318103E0EFC0EAE5F1E0A0812E
:100B5000B18112970895AAE5B1E0ED91FC91329729
:100B60000895BA93AA93089513E009E00C9407033B
:100B700030E002E00C94CE2211E00FE00C94070369
:100B800014E009E00E94070324E002E512E0089562
:100B900001E00E94CE2213E007E00E94070313E465
:100BA000089501E00E94CE2214E001E10E940703B3
:100BB00021E005E315E00E942C0327E030E00895D2
:100BC00001E00E94CE2214E00CE00E94070321E025
:100BD00001E315E00E942C0326E030E008950E9416
:100BE000070321E009E215E00E942C0324E030E035
:100BF00001E00E94CE2214E006E00E94070321E0FB
:100C00000DE215E00E942C0325E030E0089500502D
:100C100071F00A95A9F00A9549F10A95D9F10A955A
:100C2000F1F10A9509F446C00A95F1F10895FADD4B
:100C300027E00AEA12E08BDE27E009EA14E008C0A8
:100C4000F1DD24E004E412E07DDE27E000EB14E0B7
:100C500060D06ADE40DE21E000EC14E00E942C034C
:100C600029E007EB14E00E942C030895DBDD27E068
:100C700003EA12E067DE29E007EB14E00E942C0390
:100C800021E000EC14E050DE26DE27E009EA14E063
:100C900040D0E9CF42DE33D009EC14E0E4CF3DDEB2
:100CA0002ED001ED14E0DFCF0E94030324E105E81C
:100CB00014E0D9CF0E94030311E007E00E9407036C
:100CC00028E00FED14E030DEB0DD15D049F424E16A
:100CD00007EE14E02DDE0E942C0309B70F7B09BF3D
:100CE00008950E94F11E03E00E941020E0E5F1E06B
:100CF000008103950083009150010F30089504E0B6
:100D00000E94070326E009ED14E00E942C0328E06E
:100D100008950E942C0323E004E412E008950E9449
:100D2000850302E063D008951CDF8A932397802F08
:100D3000D9018D0144E648D00883188104E6109F4C
:100D4000A0190A2F4AE00E942226098319810AE08D
:100D5000109FA019A05DAA830981005D0983088105
:100D6000005D08830091FB00013069F4843059F084
:100D700000E007C0FE0110E0E00FF11F208114D059
:100D800003950330B8F3833011F423E005C00981E3
:100D900008830A81098322E08E010E941C032396A6
:100DA000A3DE08950091FA00F801EE5FFE4F208364
:100DB0000895E00FF11F24910091FA00F5CFEAEEBB
:100DC000F0E00081118148EC50E00C945E26E1993E
:100DD000FECF2EBB3FBB0DBBE29AE19A0895E1998D
:100DE000FECF0EBB1FBBE09A0DB30895005029F053
:100DF0000A95E1F10A95F1F10895F8940FDD0AC022
:100E000067D039F40091FA0010E078D0E152FF4F3A
:100E10000083FADC0091FA000A3030F50091BC0042
:100E200010E0025010402091BE0030E0021713077E
:100E30007CF072D045D00083EEEBF0E051D06CD066
:100E4000E152FF4F0083EEEBF0E000810A95E0CF26
:100E50002091BE0049D0A1F60091FA0010E0075D94
:100E60001E4F4CD02DD0D4CF78940895F8946BD0E9
:100E700078940895F8940AEF3FD014E0019F1092FF
:100E8000F500102F15FB10E010F91093F600102F4D
:100E900013FB10E010F91093F70003700093F900B2
:100EA0000DEF2AD00093BE000FEF26D012E0019F75
:100EB00004D00082118278940895EBE4F1E0089563
:100EC000E154FF4F08950250104020173107089554
:100ED0000091BE001091BC0001170895ECEFF0E006
:100EE00000810395008308950091BC0010E001503B
:100EF000104020173107089513E071CF70DF209163
:100F0000FA0030E0F901089500E32091FC0030E0A0
:100F1000F901EE5FFE4F08954091FA002091BE0066
:100F200001E210E0039F029F002D110D040F131F1B
:100F300056DFE5CFE2E1F2E00091FA0010E0E00FC9
:100F4000F11F249108958A9369DC13C04091FA003F
:100F500050E02091BE0001E210E0059F029F002DAD
:100F6000110D040F151F065F1F4FC8DFD1D000837E
:100F70004BDC0091FA000A3048F3B5DC065EF2D093
:100F8000BCD000831183AFDC0C5E1F4F28DFB5D0CF
:100F9000D1D000E0A2D000831183A5DC0B5EA0D0ED
:100FA0009CD0BFD097D0082F04FB00E000F9102F91
:100FB00000E08DD00083118396DC0A5E1F4F0FDFA7
:100FC00086D020813181B2D0000F111F00831183A0
:100FD000082F069506950370102F00E075D000834A
:100FE000118381DC095E7CD06FD09BD073D0082F39
:100FF0000370102F00E065D00083118374DC085E5D
:101000006FD05FD08ED066D0A5D0075E1F4FE7DED1
:10101000802F8F708093DE00102F12951F70177035
:101020001093DB00102F110F10E0111F1093F4002C
:101030005ADC035E97D042D00083118354DC055EF6
:101040001F4FCDDE3BD076D09BD011834CDC045EAD
:1010500047D065D03FD0082F0695069507700093BE
:10106000EE0083708093BB0075D0005E7BD021D0F2
:101070000083118338DC025E1F4FB1DE1AD05AD0D4
:101080007AD0118330DC015E2BD009D04AD022D037
:101090008695869587708093F30089910895E1EF96
:1010A000F0E0089500811181025E1F4FEDE4F1E050
:1010B0000895EFEEF0E0089500811181EAEEF0E08E
:1010C0000895ECEDF0E00895E9EDF0E00895E7ED26
:1010D000F0E00895208331830895E5EDF0E0089570
:1010E0001F4F7DDE10E008950C5E1F4F2017310763
:1010F0000895EAEEF0E000811181E3EDF0E008955B
:1011000000811181E3EDF0E00083118307E02DC140
:10111000E753FF4F0895E9EDF0E000811181ECEE17
:10112000F0E020813181200F311F089510E0020F7F
:10113000131F08952081318110E0020F131F000F4B
:10114000111F00831183082F02950F7006950370FD
:10115000102F08952091BE0001E2019F029F002DF3
:10116000110D08951F4F3BDE802F182F110F10E037
:10117000111F00E0089500E0E1EFF0E00083089522
:1011800000E0ECEEF0E000830895F89400E00093B6
:10119000FD0003C0EDEFF0E0A3DE0091FD000330A1
:1011A00008F062C0DED05BC07ED0A0D0260F371F13
:1011B000E8E9F0E0BDD077D099D0260F371F265F41
:1011C0003F4FECEFF0E0B4D01FDB0091FA000A30A3
:1011D00058F37FD02C5E3F4FE0E6F1E074D02B5EF9
:1011E0003F4FEAE6F1E06FD02A5E3F4FE4E7F1E0DF
:1011F0006AD0295E3F4FEEE7F1E065D0285E3F4FB1
:10120000E8E8F1E060D0275E3F4FE2E9F1E05BD033
:1012100043D0ECE9F1E057D0255E3F4FE6EAF1E03C
:1012200052D0245E3F4FE0EBF1E04DD032D0EAEBFC
:10123000F1E049D0225E3F4FE4ECF1E044D0215E82
:101240003F4FEEECF1E03FD021D0E8EDF1E000912E
:10125000BE00E00FF51F18D0EEEBF0E041DE1FD02E
:1012600008F098CFDBDAB1CF2AEF33E0E2EEF1E01D
:101270000BD02DEF33E000E0AADD2FEF33E0E3EEFB
:10128000F1E002D0789408950491A1CD205E3F4F03
:101290000895235E3F4F0895265E3F4F08950091C5
:1012A000BE000A3008956091FA0070E04091BE00DF
:1012B0002091FD000AE010E0079F029F002D110D14
:1012C000040F171F08950091BE00E00FF51F049151
:1012D0007EDD4091BE0050E02091FD000AE010E06C
:1012E000059F029F002D110D040F151F21E230E014
:1012F000219F300D209F202D310D089530E0219F3A
:10130000300D209F202D310D4091FE0050E00AE06D
:1013100010E0059F049F002D110D020F131F609117
:10132000FD0070E0600F711F0091020124E6089536
:101330004091BE000AE0079F049FE00DF11D00915F
:10134000FA00E00FF71F049142CDF801EE5FFE4F67
:101350002083E2E1F2E00091FA00E00FF11F249116
:10136000089500E00093BE000895F89405500E31F2
:1013700008F0E6C0F2E00F9FF001E65CFA4F05903E
:101380001490F00109944ADA0091FA000A3008F04A
:10139000D7C006D10091FA00F1D0008118DD34DA0F
:1013A000F3CF3CDA0091FA000A3008F0C9C0F8D057
:1013B000265F3F4F0091FA00DAD0008108DD24DA81
:1013C000F1CFE4D02C5E3F4F98DE8BDADBD064DFC8
:1013D0005F7793DE00811181159507950078052BC5
:1013E000AEC0D4D02B5E3F4F78DE7BDACBD054DF5B
:1013F0005F7973DEB0D0007EF2CFC8D02A5E3F4F57
:1014000066DE6FDABFD048DF5F7E61DEA4D015955F
:101410000795007FE4CFBAD0295E3F4F55DE61DAF1
:10142000B1D03ADF537F50DE0081118146E00E9447
:1014300040260C7FD4CFAAD0285E3F4F42DE51DA3F
:10144000A1D02ADF5C7F3DDE1181012FC8CF9ED065
:10145000275E3F4FE4EFF0E0008100FB00E007F97A
:101460001091DB001295107F100F0091DE00010F2C
:1014700066C08CD0255E3F4F21DE33DAA0D009DF75
:101480000F771CDE65D061D04078402B042F57C009
:101490007DD0245E3F4F56D024DA91D0FADE0F790A
:1014A00051D056D052D051D050D0407EEECF1BDA22
:1014B00086D0EFDE007E4091EE00440F440F109185
:1014C000BB00140F102B012F3AC060D0225E3F4F9B
:1014D000F0DD07DA005E74D0D9DE0F77EADDD2CF17
:1014E00055D0215E3F4FDBDDFCD9005E69D0CEDEFA
:1014F0000F79D5DDD6CFF7D9005E62D0C7DE007E8A
:101500001091F300110F110FDDCF2FEF33E0D5DC79
:10151000FEDA15C02AEF33E00091F50010E4019FD8
:101520000091F6000295007F000F00291091F7004E
:10153000110F110F110F102B0091F900012B47DC37
:1015400078940895ECEEF0E0089555954795089548
:101550004081518108950081118115950795159558
:1015600007951595079508950091FA0010E0F80188
:10157000E753FF4F08950091FA0010E0F801E1549D
:10158000FF4F0895065E1F4F2ADC502F0091BE00CA
:1015900010E021E230E0219F209F202D310D0895A1
:1015A0004091FA0050E00091BE0010E021E230E0EE
:1015B000259F209F202D310D240F351F0895035E98
:1015C0001F4F0DDC4091BE0050E021E230E0259F2E
:1015D000249F202D310D089530E0259F209F202D40
:1015E000310D409103010AE010E0059F049F002D9A
:1015F000110D020F131F209104010895E7EDF0E093
:101600000081118148EC50E00E945E260093FD00AD
:10161000E7EDF0E00081118142E050E00E945E269B
:101620004091FD0050E024E630E0259F249F202DCE
:10163000310D021B130B4AE00E945E260093FE0050
:10164000E7EDF0E00081118142E050E00E945E266B
:101650002091FD0014E6219F00192091FE001AE060
:10166000219F0019005D0093FD00EEEFF0E0008186
:10167000005D0083E7EDF0E00081118148EC50E06F
:101680000E945E26005D1F4F24E608954A9269DAA3
:101690009A938A93402E80E090E080931D01789485
:1016A00004E009BF0E94030308C0008100FD03C0DD
:1016B0000E949A1EC4D8892F90E101E0401611F0D3
:1016C0000C948219882309F065C00E94CB1B0091FD
:1016D0001D010E94E21A0E94551A34C00091FA00BE
:1016E000073028F4EBE0F2E027DC0E94A41A0E9405
:1016F000461A51F4ECE1F2E01FDC54DBE6E2F2E0E2
:101700002ADE0E949D1A81E00E94421A49F4E6E214
:10171000F2E012DC0091FA0018DE0E949D1A8EE0C1
:101720000E943E1A49F406DC3DDBECE1F2E013DEF8
:101730000E949D1A80E190E067D80091FA000A307B
:1017400068F27DD80E94211A79F00E941D1A61F07A
:101750000E94151A0E940D1A11F40E94091A0E9483
:10176000051A81F75BD8E9CF0E94211A41F480E085
:1017700080931D010E940D1A11F40E94C61B0E9445
:101780001D1A21F40091240100931D010E94BF1B2A
:1017900000935101813009F095C00E94CB1B10913C
:1017A000F9000AE0109F002D065F0093BC000E9424
:1017B000B91B00911E011091BC00011719F4009192
:1017C0001E0102C00091BE000E948D1A0E94551A8F
:1017D00001C035D80E94211A09F460C00E941D1A68
:1017E00009F45CC00E94171A11F40E94091A0E94A1
:1017F0000D1A11F40E94091A0E94051A59F7009156
:1018000024010093BE0000E0F1DA62DB29F40091CC
:10181000BC000A950093BE000E940E040DC00E94F9
:101820001A1B0E94021A20830E94971A20810E948C
:101830009D1A82E00E9404040091FA000A3048F6E2
:101840000091FA00073028F4ECE1F2E075DB0E9429
:10185000A41A0E944A1A61F46DDBA4DA0E94971A56
:101860000E941C1BE45FFE4F208380E191E0E2CFE9
:101870002091240130E038DB0091FA0010E0F801FB
:1018800071F60E941A1B0E94021A2083E2E1F2E024
:101890000091FA00E00FF31F2491C9CF0E94211A92
:1018A00041F480E080931E010E940D1A11F40E9401
:1018B000C61B0E941D1A21F40091240100931E01F1
:1018C0000E94BF1B8E3009F0BDC00E94CB1B09B324
:1018D0000C700C3011F004E001C003E00093BC0078
:1018E00000911F010E948D1A0E94551A02C00E9489
:1018F0001F040E94211A09F47CC00E941D1A09F4D9
:1019000078C00E94171A11F40E94091A0E940D1A39
:1019100011F40E94091A0E94051A59F70E940E0438
:1019200017C008DB3FDA0E94FB1915DD0E949D1AE3
:1019300080E19EE00E943A1A49F4FCDA33DA0E9410
:10194000FB1909DD0E949D1A80E19EE00E940404BB
:101950000091FA000A3058F60091FA00073028F496
:10196000E6E2F2E0E9DA0E94A41A0E94461A51F473
:101970000E94FB19E1DA16DAEBE2F4E0ECDC0E94FB
:101980009D1A81E10E94421A51F4EBE2F4E0D4DAAC
:1019900009DAE1E2F4E0DFDC0E949D1A84E20E94B1
:1019A0003E1AA1F40091BC000430E1E2F4E00091A1
:1019B000FA0010E021F4FDD9E3E5F4E003C0F9D921
:1019C000E2E1F2E0C8DC0E949D1A80E00E94361A33
:1019D00009F0B0CF0091BC00043009F0A2CFE3E5DC
:1019E000F4E0AADA0091FA00B0DC0E949D1A8DE0C2
:1019F000A1CF0E94211A41F480E080931F010E9430
:101A00000D1A11F40E94C61B0E941D1A79F40E943F
:101A10003E1A61F40E94B91B00931D0106E0F7D83D
:101A2000B4DB9FDC0E9403030E941F040E941D1A66
:101A300039F40E943E1A21F00091240100931F0105
:101A40000E94BF1B8D3009F0BCC00E94CB1B0091CF
:101A500023010E94E21A0E94551A5AC00091FA000E
:101A6000073028F4E3E5F4E067DA0E94A41A0E9444
:101A7000461A71F4EDE5F4E05FDA94D9E7E6F4E0B4
:101A80006ADC0E949D1A0E94F61985E210935201A9
:101A90000E94421A71F4E7E6F4E04EDA83D9E1E7F6
:101AA000F4E059DC0E949D1A0E94F6198EE0109312
:101AB00052010E943E1A19F50E942C1B31F4E1E7F5
:101AC000F4E03ADA6FD9109352010E94281B89F48E
:101AD0000091FA00002319F401E00E945B1F0091BD
:101AE000FA00033020F0EBE7F4E026DA5BD90E943D
:101AF000F219EDE5F4E020DA0E949D1A8DE00E94D3
:101B000004040091FA000A3008F4A8CF0E941F04D0
:101B10000E94211A61F10E941D1A49F10091F700FB
:101B20000093F80001E00093F7000E94171A11F4E7
:101B30000E94091A0E940D1A11F40E94091A0091BC
:101B4000F8000093F7000E943E1A59F40E94EE1923
:101B500040F003E0009324010E94551A01E0009335
:101B6000FC000E94051AA1F60E940E04CACF0E9432
:101B7000211A69F40E94251A09F480E00E94B51B1D
:101B8000009352010E940D1A11F40E94C61B0E947C
:101B90001D1AA9F40E94461A51F401E00E94501A3D
:101BA0000E94B11B0093FB0000932B0106C00E9412
:101BB000421A19F400E00E94501A0E94B51B0E94BC
:101BC000BF1B823009F087C00E94CB1B0E94E51A20
:101BD000009122010E948D1A0EE001C007E00093DF
:101BE00056010E94211A09F45CC00E941D1A09F4D2
:101BF00058C00E94171A11F40E94091A0E940D1A67
:101C000011F40E94091A0E94051AE9F50E940E04B7
:101C100034C00091FA00073048F40091FA0010E057
:101C2000F8010E941A1BEA5EFE4F20830E94461AAA
:101C300051F4E0E3F2E080D9B5D8EAE3F2E08BDBDF
:101C40000E949D1A83E00E94421A49F4EAE3F2E0FE
:101C500073D90091FA0079DB0E949D1A84E00E94FA
:101C60003E1A49F467D99ED8E0E3F2E074DB0E94A3
:101C70009D1A80E192E00E9404040091FA000A306B
:101C800040F20E941F040E94A5053CF000811181D2
:101C90000B3F0E94211B0CF4A1CF01E00E94391BD5
:101CA000A0CF0E94211A81F481E00E94EA1909F470
:101CB00080E000E00E94BD1B0E9418040E940D1AE3
:101CC00019F483E0109353010E941D1A21F400912E
:101CD00024010E94BD1B813109F0B9C00E94CB1BB9
:101CE000009120010E948D1A04E00093BC00009135
:101CF000F5000093FD000E94551A59C00091FA00AA
:101D0000073028F40E94FB1917D90E94A41A0E94D8
:101D1000461A61F4EBEDF3E00FD944D8E7ECF3E0B9
:101D20001ADB0E949D1A1093F5008EE00E94421A61
:101D300061F4E7ECF3E000D935D8E5EEF3E00BDB36
:101D40000E949D1A01E00E94E6190E943E1A61F469
:101D5000E5EEF3E0F1D826D8E1EDF3E0FCDA0E94FD
:101D60009D1A02E00E94E6190E94361A59F4E1ED2C
:101D7000F3E0E2D80091FA00E8DA0E949D1A03E04D
:101D80000E94E6190E943A1A49F4D4D80BD8EBED18
:101D9000F3E0E1DA0E949D1A80E191E10E940404DF
:101DA0000091FA000A3008F4A9CF0E941F040E9493
:101DB000211A99F00E941D1A81F00E94171A11F43D
:101DC0000E94091A0E940D1A11F40E94091A0E9419
:101DD000051A69F70E940E04E3CF0E94211A69F4E4
:101DE0000E94731A0E94AD1B0E94251A09F480E01C
:101DF0000E940D1A11F40E94C61B0E941D1A29F59B
:101E0000009157010023E9F40091F500023021F020
:101E10000091F5000330A9F40E94030312E00E9430
:101E2000150424E107EF11E00E9498040E942C039E
:101E30000E94DF190E94641AE9F70E9403030E94BE
:101E4000731A0E94AD1B0E94521A0E94BF1B84305D
:101E500009F0E8C20E94CB1B009121010E948D1A5B
:101E60000BE00093BC0001E00E94F60600E0009346
:101E70002B010093FB000E94551A02C00E941F0410
:101E80000E94211A09F4B2C20E941D1A09F4AEC2BE
:101E90000E94171A11F40E94091A0E940D1A11F4D7
:101EA0000E94091A0E94051A19F00E94EE1941F7C2
:101EB0000E940E041FC0E1E4F3E03ED80E94D20667
:101EC0000091FA00093011F40E94A91B42DA0E9425
:101ED0009D1A83E2009124010B3051F42BD80E940B
:101EE000D206EFE8F2E037DA0E949D1A80E194E032
:101EF0000E9404040091FA000A3000F60091FA00F2
:101F0000073028F4EAE3F2E017D80E94A41A0E94EE
:101F1000461A21F00E94421A09F041C00E94CF1BCC
:101F200041F40E94E21B11F400E001C001E00093C3
:101F3000FB000E94B11A0091240161F4002339F4DE
:101F4000EFE8F2E00E949C070E94D20618C0E9E97F
:101F5000F2E0F8CF00230091FA0010E0F80119F444
:101F60000E94600701C0D4D80E941C1B0E94021A64
:101F700020830091FA00093011F40E94A91B0E94ED
:101F8000461A39F4E9E9F2E0E6D90E949D1A83E1A4
:101F900006C0E1EBF2E0DFD90E949D1A84E10E94C5
:101FA0003E1A81F00E94361A69F00E943A1A51F0E6
:101FB0000E94321A39F00E942E1A21F00E942A1A29
:101FC00009F054C101E00093E9000E94EE1941F4C8
:101FD0000E94E21B11F400E001C001E00093FB004D
:101FE0000E94B11A09F050C00E943E1A31F4E1EB90
:101FF000F2E00E949C070E94D2060E94361A31F439
:10200000EBEBF2E00E949C070E94D2060E943A1A73
:1020100091F40E94DB1919F4ECECF2E008C00E9484
:10202000D71919F4E5E5F3E002C0E3E7F3E00E9415
:102030009C070E94D2060E94321A91F40E94DB197A
:1020400019F4E6EDF2E008C00E94D71919F4EFE5A3
:10205000F3E002C0EDE7F3E00E949C070E94D20685
:102060000E942E1A31F4E1EFF2E00E949C070E94D8
:10207000D2060E942A1A09F099C0EBEFF2E00E9402
:102080009C070E94D20692C00091FA00002309F03A
:1020900044C00E94B2040E943E1A21F40E948505A9
:1020A0000E9482050E94361A19F417D80E94A105D1
:1020B0000E943A1A89F40E94DB1911F408D808C06A
:1020C0000E94D71919F40E945E0802C00E945908A4
:1020D0000E9487050E9482050E94321A79F40E94AC
:1020E000DB1919F40E94640807C00E94D71911F483
:1020F00029DA02C00E944F080E94A1050E942E1AF0
:1021000029F40E94591A46DA0E94111A0E942A1ACA
:1021100021F40E9461080E94A1050091FA00033099
:1021200011F40E94C9190091FA000430C8F10E940C
:102130003E1A19F00E943A1AA9F40091FA000430EC
:1021400021F40FED009306010DC00091F60000236D
:1021500019F4EFEEF3E002C0E9EFF3E00E949C0710
:102160000E94D2060E94361A31F00E94321A19F0EB
:102170000E942A1A61F40E94960519F4E3E0F4E043
:1021800002C0EDE0F4E00E949C070E94D2060E948B
:102190002E1A31F4E7E1F4E00E949C070E94D20677
:1021A0000091FA00093011F40E94A91B0E943E1A06
:1021B00039F4EBEBF2E00E949C070E949D1A85E146
:1021C0000E94361A99F40E94DB1919F4ECECF2E043
:1021D00008C00E94D71919F4E5E5F3E002C0E3E76F
:1021E000F3E00E949C070E949D1A86E10E943A1A21
:1021F00099F40E94DB1919F4E6EDF2E008C00E94A0
:10220000D71919F4EFE5F3E002C0EDE7F3E00E941F
:102210009C070E949D1A87E10E94321A99F40E943D
:10222000DB1919F4E0EEF2E008C00E94D71919F4A6
:10223000EBE4F3E002C0E9E6F3E00E949C070E94B1
:102240009D1A88E10E942E1A39F4EBEFF2E00E9409
:102250009C070E949D1A8AE10E942A1A39F4E5E03F
:10226000F3E00E949C070E949D1A8BE100912401DB
:10227000063009F064C00E94CF1B41F40E94E21BAB
:1022800011F400E001C001E00093FB000E94B11ACC
:102290000091BB0091F4013039F4E0EEF2E00E94CD
:1022A0009C070E94D20645C00E94D71919F4EBE49E
:1022B000F3E0F5CFE9E6F3E0F2CF013089F40091E5
:1022C000DB00002319F4E3EBF3E029C00091DB000D
:1022D000013019F4E9EAF3E022C00091DB0018C0F4
:1022E0000E94D71959F40091EE00002361F3009188
:1022F000EE00013079F30091EE000AC00091F30086
:10230000002309F30091F300013021F30091F30061
:10231000023019F4EFE9F3E002C0E5E9F3E00E94CE
:102320009C070E94D2060091FA00093011F40E9425
:10233000A91BE1EFF2E00FD80E949D1A89E10091FC
:102340002401093071F50E94CF1B41F40E94E21B69
:1023500011F400E001C001E00093FB000E94B11AFB
:1023600039F4E5E0F3E00E949C070E94D20612C017
:102370000E94960519F4EFE0F3E002C0E9E1F3E012
:102380000E949C070E94D2060091FA00093011F4C5
:102390000E94A91BE3E2F3E00E94AB090E949D1A90
:1023A0008CE1009124010A3009F094CD0E94CF1BEA
:1023B00041F40E94E21B11F400E001C001E000932F
:1023C000FB000E94B11A39F4E3E2F3E00E949C079B
:1023D0000E94D2067BCDEFD719F4EDE2F3E06DCD8C
:1023E000E6D709F068CDE7E3F3E067CD0E94211A54
:1023F00061F400E00093210182E0ECD709F480E071
:102400000E940D1A11F40E94C61B0E941D1A21F48D
:1024100000912401009321010E94BF1B0093FB0047
:102420000093FC00833119F0843109F0B2C00E949E
:10243000F81B01E00093FF000E94551A02C00E94A1
:102440001F04FFD709F46DC0F8D709F46AC0EFD7AD
:1024500009F4DFD7E2D709F4DCD7D7D791F70E9488
:102460000E040DC00E94311B03950E94301B0C32DC
:1024700021F40DE20E94850700830E94040400916C
:10248000FA000A30E0F60091FA00073058F4833180
:1024900019F4EFE8F2E002C0E9E9F2E00E949C07DB
:1024A0000E94A41AF3D7A9F40E942C1B59F46BD7ED
:1024B00019F40E94600702C00E9488080E941C1B39
:1024C000A1D72083E5E8F2E00E949C070E949D1AB4
:1024D000D4CFD8D70091FA00B1F4093071F60E9438
:1024E000C21B0E943D1B003221F40FE70E948507AA
:1024F00003C00E94311B0A950E94301B0C3209F068
:10250000BCCF0BE2B7CF093009F0B7CF0E94C21B96
:102510000E943D1B0F3709F0A5CF00E20E948507FE
:10252000A4CF8FD751F40E94A51B84E053D709F4A0
:1025300080E073D711F40E94C61B7FD741F50E943B
:102540006E070091FC000A3011F50E94B11B009348
:10255000FA0007C057D70E941C1B0E9488080E94DF
:1025600003040091FA000A3040F40DD799F74AD7D6
:102570000E941C1B0E946007F2CF833111F405E01A
:1025800001C006E00E94B5090E94A51B84E00E94DC
:10259000BF1B853169F0863159F0873149F08831A8
:1025A00039F08A3129F08B3119F0853209F0E2C314
:1025B0000E94F81B01E00093FF000E942C1B29F4ED
:1025C000C8D600930301009304016FD702C00E9494
:1025D0001F0437D709F416C330D709F413C327D71C
:1025E00009F417D71AD709F414D70E942C1B09F441
:1025F00010C1873109F06DC00E949605A5D630E064
:1026000059F40E944D1B213106E130076CF003E3C1
:102610000093020102E307C00E944D1B91D624F0F3
:1026200002E30093020199D6C6D6D1F50E947D0837
:102630000E94E1060093FD000E9485057CD60E9461
:10264000E60AB8D70E94850590D7005D00837CD646
:102650000E94CA0A4091030150E00AE050D7A091BD
:102660000401B0E0A00FB11F0E947D08008111811C
:1026700048EC0E945E26005D1F4F24E60E94770909
:102680004091FE0050E00AE010E039D72091FD00B3
:102690000E945C1BA217B3071CF40E947D0878D728
:1026A00086D659F40E94FE0A0E947E090E94EC0A16
:1026B0000E945C1B3DD60CF469D771D651F40E9480
:1026C000FE0A0E947E090E94EC0AF6D731D60CF46D
:1026D0005DD7883109F040C00E949605E9F56BD6B8
:1026E00051F432D60E94CA0ADCD7293207E13007FA
:1026F00014F006E339D65BD6A9F4E2D74091030182
:1027000050E0420F531F0E94640800811181040FA2
:10271000151F0053104066D72CF00E9484070083D9
:102720000E941F043CD6C1F4CBD7009103010E9444
:1027300096080E9464080E9491080E94A20A0081E3
:102740001181020F131F005310404CD72CF00E9430
:10275000840700830E941F04853109F043C0F4D52B
:102760000E94CA0A9ED72230ECD51CF4F2D505E3AC
:10277000F4D521D659F40E94FE0A0E947E090E94D7
:10278000EC0A9AD7D5D524F501D722C00E94DF06DE
:102790000093FD000E945E080E948705CCD50E9430
:1027A000E60A08D70E945E080E948705DED6005D13
:1027B00000830E94DF06005D1F4F24E60E947E0911
:1027C0000E94EC0A79D7B4D51CF40E945E08E0D6CA
:1027D000BBD50E94CA0A65D7B3D524F002E30093A3
:1027E0000201BBD58A3149F4AFD50E94CA0A59D734
:1027F0002533A7D514F001E3B7D5853251F4A4D51C
:102800000E94CA0A4ED7253C06E1300714F005E3C2
:10281000ABD5FBD509F0DDCE0E940E0405C021D753
:10282000039500830E9404040091FA000A3008F026
:10283000CECE0091FA00073008F045C0853129F46A
:10284000E1EBF2E00E949C077FD6863129F4EBEBA6
:10285000F2E00E949C0778D6873179F4ACD519F460
:10286000ECECF2E007C0A3D519F4E5E5F3E002C013
:10287000E3E7F3E00E949C0767D6883179F49BD5A3
:1028800019F4E6EDF2E007C092D519F4EFE5F3E0B4
:1028900002C0EDE7F3E00E949C0756D68A3129F486
:1028A000E1EFF2E00E949C074FD68B3129F4EBEF69
:1028B000F2E00E949C0748D6853229F4EDE5F4E069
:1028C0000E949C0741D6E2D509F0A3C0C5D609F005
:1028D00091C00091FA00002309F048C001E0009384
:1028E000FB000E94B204853121F40E9485050E94FC
:1028F0008205863121F40E946D080E94A10587316E
:1029000081F459D519F40E94670807C050D519F40D
:102910000E945E0802C00E9459080E9487050E941A
:102920008205883171F447D519F40E94640807C004
:102930003ED519F40E94A20A02C00E944F080E94CC
:10294000A105853239F40E945D070E94A10500E3CC
:10295000009304018A3121F4ACD50E94CA0A61D5E2
:102960008B3121F40E9461080E94A1050091FA00B8
:10297000033009F40ED50091FA000430D8F1853106
:1029800011F08731A9F40091FA00043021F40FED21
:10299000009306010DC00091F600002319F4EFEE3C
:1029A000F3E002C0E9EFF3E00E949C070E94D20628
:1029B000863121F0883111F08B3161F40E94960547
:1029C00019F4E3E0F4E002C0EDE0F4E00E949C07BB
:1029D0000E94D2068A3131F4E7E1F4E00E949C07BC
:1029E0000E94D206853231F4EBE7F4E00E949C07A6
:1029F0000E94D206E5E8F2E00E949C079ED58A314B
:102A000009F010CF21D609F00DCF07E00093560151
:102A100009CF38D50091FA0009F082C0093009F0D9
:102A200001CFB0D619D609F06EC0873169F4009194
:102A30000201003321F403E30093020105C0E2E048
:102A4000F1E000810A950083853151F416D60033F8
:102A500021F402E30E94850702C003D60A95008391
:102A6000863121F0883111F08B31A9F506D600337B
:102A700021F409E30E94850702C0F3D50A9500837B
:102A8000883149F50E94960531F595D439F4E9D598
:102A9000063320F006E30E948507008388D461F4A2
:102AA0000091FC0058D52CD61F4FA017B10724F079
:102AB00027D60E948507008372D469F40091FC0038
:102AC00010E049D52BD61F4FA017B10724F026D60A
:102AD0000E94850700838A3151F4CFD5003321F459
:102AE00001E30E94850702C0BCD50A9500838532A8
:102AF00051F4C3D5023321F405E30E94850702C0D7
:102B0000B0D50A950083A8D509F48CCEB6D500338C
:102B100021F409E30E94850784CEA3D50A9581CECE
:102B2000093009F07FCE2ED697D509F062C08731E3
:102B300051F400910201033311F40BD404C0E2E01C
:102B4000F1E00E947007853149F497D5023319F4FA
:102B50000E94840702C085D503950083863121F049
:102B6000883111F08B3171F588D5093319F40E9441
:102B7000840702C076D503950083883119F50E9439
:102B8000960501F518D431F46CD5073318F00E947E
:102B9000840700830CD451F4B3D51F4F0E948507DE
:102BA00020810217130714F429D40083F8D351F4B9
:102BB000B5D51F4F0E94850720810217130714F413
:102BC0001DD400838A3149F458D5013319F40E9489
:102BD000840702C046D503950083853251F44DD554
:102BE000053321F402E30E94850702C03AD503951C
:102BF000008332D509F416CE40D5093309F00FCE43
:102C000000E388CF1ED461F4A0D5853211F48DE0A5
:102C100001C084E0DFD309F480E0FFD309F4B6D526
:102C20000CD409F0A6C00E946E07853229F40CD599
:102C300019F403E00093FC000091FC00033009F05C
:102C400098C08FD53DD5009104010E94960800538D
:102C50001040D5D4853111F40E948008863149F4A2
:102C60000E9491050E946D080083118309E00E9473
:102C7000B509873189F59FD351F40E9491050E94CF
:102C800067080083118308E00E94B50925C08FD32F
:102C90000E94910579F02DD50E945908008111817B
:102CA000000F111F0E945E08B9D4B4F40E945908A5
:102CB000008111811DD40E945E0800811181000FE6
:102CC000111F0E947D08AAD43CF40E945E080E9455
:102CD000800802E0009321018831D9F46CD341F4DB
:102CE0000E9491050E946408008311830AE00FC0CE
:102CF0005ED30E94910531F40E94A20A00831183E1
:102D00000EE105C00E944F080083118301E20E947A
:102D1000B5098A3191F4E0E0F1E0A081B1811A9720
:102D200014F400E005C0008111814AE00E94E4062D
:102D30000093DE000CE00E94B5098B3149F40E943B
:102D400091050E946108008311830BE00E94B50980
:102D5000853249F40E9491050E945D07008311832A
:102D60000DE00E94B509F1D4853211F48EE001C066
:102D700084E005D58C3139F0833229F0893119F09E
:102D8000843209F030C207D58C3149F401E0009358
:102D9000BC000091F400C1D30091F4002BC0843238
:102DA00039F413D40091F900B8D30091F90022C08E
:102DB0008931C9F403E00093BC00FDD231F40091E5
:102DC000DB00ABD30091DB0015C0F1D231F40091F0
:102DD000EE00A3D30091EE000DC00091F3009DD34F
:102DE0000091F30007C0F1D30091BB0000932401D0
:102DF0000091BB000093FC0058D302C00E941F0446
:102E000020D309F4E1C019D309F4DEC010D309F4CA
:102E100000D303D309F4FDD2F8D291F70E940E0437
:102E200009C00093F300E5E8F2E00E949C0779D323
:102E30000E9403040091FA000A3000F70091FA00A2
:102E40000730F0F48C3119F4E5E0F3E016C0843279
:102E500019F4EBE2F4E011C0893169F4ACD219F451
:102E6000E0EEF2E00AC0A3D219F4EBE4F3E005C00F
:102E7000E9E6F3E002C0E3E2F3E00E949C0764D3DA
:102E800005D3A9F58C3149F4EFE0F3E00E949C07EB
:102E90000E94D2061093F400C6CF843249F4E5E3D1
:102EA000F4E00E949C070E94D2061093F900BBCF69
:102EB000893199F4E3EBF3E00E949C070E94D2066B
:102EC0007AD219F41093DB00AECF71D219F41093BB
:102ED000EE00A9CF1093F300A6CFEDE2F3E00E943D
:102EE0009C070E94D20601E00093BB009CCFCAD28F
:102EF000A9F58C3151F4E9E1F3E00E949C070E94AE
:102F0000D20601E00093F4008ECF843251F4EFE357
:102F1000F4E00E949C070E94D20601E00093F900B1
:102F200082CF893199F4E9EAF3E00E949C070E947C
:102F3000D20641D221F401E00093DB0074CF37D2F6
:102F400001E019F40093EE006ECF6BCFE7E3F3E0FE
:102F50000E949C070E94D20602E0C6CF8FD211F5D4
:102F6000843241F4E9E4F4E00E949C070E94D20616
:102F700002E0D4CF893171F4EFE9F3E00E949C07BD
:102F80000E94D20618D211F402E0D6CF10D202E08D
:102F9000C9F247CFE1E4F3E00E949C070E94D20609
:102FA00003E0A2CF893109F03ECFE5E9F3E00E94CA
:102FB0009C070E94D206FFD111F403E0BDCFF7D1E8
:102FC00003E009F02ECFBECF3CD269F58C3129F455
:102FD0000091FC000093F4001FC0843231F4009192
:102FE000FC000093F9008EE018C0893189F4E3D128
:102FF00029F40091FC000093DB000EC0D8D10091B1
:10300000FC0019F40093EE0007C00093F30004C025
:103010000091FC000093BB0084E0DCD109F480E067
:10302000FCD109F4B3D309D209F0DCC08C3109F02A
:103030004BC0EAD2B9F40E94670840D21CF018D302
:1030400008E09BD10E945E0839D21CF011D30DE13B
:1030500094D10E94590832D2ACF10CED10E04BD360
:1030600004E02EC00E948B080E944F08B7D254F192
:103070000E94640800811181093512071CF061D398
:103080000AE005D30E94A20A008111810E9464080F
:103090000E949108293502E030072CF00E94C008F8
:1030A00001830EE1F4D20E944F080E948D080E9415
:1030B000640894D23CF00E94BB08018327D205E04B
:1030C000009321010CE08BC08432A1F4EBD18EE09F
:1030D0000091F900002339F40E944F0908F482C0DE
:1030E0000E94B1097FC00091F900013009F07AC057
:1030F00010D2F4CF893139F45ED121F358D109F4DB
:103100006DC002E26CC00E94960551F550D189F461
:103110000E946408008111810C3221E012074CF0FA
:1031200008E512E080D200831183B3D20EE10E9441
:10313000B50935D1A9F40E948B08203901E0300788
:103140007CF008E512E00E9464086DD22081318194
:10315000021B130B0E944F08008311839AD2D6D111
:1031600026D1A9F40E9467080E945C0857D22CF46B
:103170000E9467080E948705BBD10E9479084ED241
:1031800034F40E945E080E9487050E94820807D1DD
:1031900029F50E946708008111810E9459083ED2DA
:1031A0002CF40E9467080E948705A3D20E94590848
:1031B0000E945C0833D22CF40E9459080E948705B3
:1031C00097D10E9479082AD24CF40E945E080E948E
:1031D00087050E94820802E0009321010FE10E940E
:1031E000B50984E0CCD2833009F080C000E30093BD
:1031F000520101E015D70E940E0408C000E00E94B1
:103200007F07E35EFE4F00830E9404040091FA00F2
:103210000730A0F32DEF33E00091BE000E94E706D7
:1032200001E00E94F606B7D2969801E000932501CE
:1032300084D20E94CB02E8D109F0E4D2FED009F09A
:1032400091D301E00093FC0005C0073009F04BD496
:103250000E946E070091BB001091FC0001170091C5
:10326000560198F7073009F0DCD40E94A5050CF050
:1032700033D15FD259D0F1F360D202E0D1D6DDD0A4
:10328000E9F043E0FFD101E00E9407060FE011C022
:1032900000915701013011F40E944324A2D540D07F
:1032A00011F44BD2C2D00E94A50514F435D019F404
:1032B00007E000935601C1D059F775D52AD0008197
:1032C00011810536BED12CF4969A209325010E94D7
:1032D000CB0247D20FE00093560182E001E0009359
:1032E000240159D20093520100935301803111F00F
:1032F0000C945D0B0AD000FD02C00C94550B53D505
:103300000C945A0B66D149900895EFE4F1E00081E6
:103310000895E4E4F1E00895009155010130089525
:10332000009126010130089500912601002308959F
:103330006217730708954091FD0050E024E6089558
:103340002D3A05E1300708950091020110E024E6CE
:10335000089500E30093020108950093030100E340
:10336000009304010C941F040093020100E30093F6
:103370000301009304010C941F040E94B50904E0AA
:1033800000932101089583310091FA0010E0F801C3
:103390000895E2EFF3E00491009305010895009190
:1033A000BB00033008950091DB0000935C010091A5
:1033B000BB00023008950091BB000130089541E048
:1033C00020ED37E000E41FE10C94A3220093F50008
:1033D0008EE00895009151010130089500912B0174
:1033E0000230089501E300935201089510932B01D8
:1033F0001093FC000895EDEBF3E0089500E32091B5
:10340000FC00F901EE5FFE4F08950E94EB230130AE
:1034100008950DE000935601089500915301013085
:10342000089503E00C949406DCD403E0F9C503E0AE
:10343000F7D50091510101300895009156010730F0
:103440000895009156010D3008958EE000915101CC
:10345000013008950091240108300895009124015D
:10346000073008950091240105300895009124014A
:10347000033008950091240104300895009124013F
:103480000230089500912401013008950091240133
:1034900000230895009124011091BC0001170895A4
:1034A0000093F7000EE00C94B5090EE0009356016E
:1034B00008950091DE0010E02AE008950081118156
:1034C000093B21E012070895EDE2F1E0008111814E
:1034D00000342FE112070895008111810F5F1F4F03
:1034E0000083118308950091FD000093F500089575
:1034F000EAEEF0E0008311830DE10C94B509059F1D
:10350000049F002D110D020F131F089501E20C946A
:10351000B5090091BE00043108950395009324017C
:1035200008950091FA00F801E45FFE4F08950091BC
:10353000FA00F801E152FF4F08950091FA00F801F6
:10354000E45FFE4F208308950091FA00F801EA5EDF
:10355000FE4F20830895F801EE5FFE4FA081B0E09A
:1035600008950091FB00002308952091FD0014E6CA
:10357000219F00192091FE001AE0219F0019005D93
:103580000093FD00EEEFF0E000810895E7EDF0E03C
:103590000081118148EC0E945E26005D00930201CB
:1035A0000091FE00009303010091FD0000930401CF
:1035B0000C941F04021B130B4AE00E945E2600932A
:1035C000FE00089503950093240102E00093BC00DF
:1035D000089589919991A991B991089500811181D6
:1035E000020F131F093522E012070895008311838B
:1035F00005E300935201E7EDF0E000811181E0E086
:10360000F1E00083118308950091F40001300895E2
:10361000E4E4F1E000811181E0E0F1E0208131811A
:1036200002171307089520813181021B130BECEE62
:10363000F0E00895E154FF4F20810091FA00F80175
:10364000089520E0120708950091FC0002300895CB
:103650000091FC00013008950091FC0000230895C2
:1036600000830091FC00F801EE5FFE4F0081089599
:103670000CED10E00083118308950091FC0010E030
:10368000F2CF41E020ED37E000ED17E05CC70E948B
:10369000B50905E0009321010895219F209F202D69
:1036A000310D409103010AE0019F049F002D110D8F
:1036B000020F131F2091040130E0200F311F0895E5
:1036C000E0910201F0E0F09704E610E00F9F100D8A
:1036D0000E9F002D110DE0910301F0E0F0972AE01C
:1036E00030E02F9F300D2E9F202D310D200F311FE8
:1036F0000895EFEEF0E00083118300E20C94B50929
:1037000008E512E0E9EDF0E020813181021B130BA6
:1037100044E650E00E945E26005D089508E512E050
:10372000E9EDF0E020813181021B130BECEEF0E0BB
:10373000EBCF06EF0CBD02EC0DBD00E000932601BF
:10374000089500E000830183089500E00093FF00E6
:10375000089500E00093FB00089500E0009320012D
:10376000089500E00093FC00089500E00093230119
:10377000089500E000931F010895009322010FE0D7
:103780000093560100E000932401089583E000E0D7
:1037900000935301089500E000935101089500E063
:1037A0000093E90000912B01023008950FE000938F
:1037B000560181E000E000932B0106EF0CBD02EC06
:1037C0000DBD089500E000932B010091FB00013036
:1037D00008950091BC000093FE000091BE000E5FB2
:1037E0000093BC0000E00E94F60601E00C94F6068F
:1037F00000E00093510101E00093240102E00093F6
:10380000BC000895EFDDCFD20AE8B2D602E053D370
:103810000E947D08F2DE9DD00E947F050083018317
:1038200084D01093260110932C017CD01083118337
:103830000091BF000F34E1F40091C0000035C1F4E5
:103840000091C1000435A1F40091C200093481F453
:103850000091C3000D3461F40091C400093441F4B7
:103860000091C5000A3521F401E00093550102C022
:10387000109355010FE0009356010E940E0404C0FE
:10388000E3EAF2E00E94F8030091FA000730C0F387
:103890000E94CF0449DDF1F350DF10E00E947F0564
:1038A000008301830091BD00013059F4009156015D
:1038B0000B3029F402E0EAE5F1E000831183109374
:1038C000BD0030D009DE00915701013009F4DBD78B
:1038D000ACDD87D20E94F22497DE09F436D0009145
:1038E00056010E3019F484D637D003C00FE0009390
:1038F00056010E949105085210400BDD8FDE0CF03E
:103900002BD010D000811181083C9BDE2CF00E944E
:103910007F052083218319D000912C01063008F403
:10392000ACCF0895EDE5F1E0089547CFE9E2F1E08D
:103930000081118101501040008311830CE310E0DD
:10394000E7E2F1E000831183089506E000932C0183
:10395000089500E010E0089500E0EDE5F1E0008357
:10396000018308950E94B1053DDD43E08BDE02E056
:103970000E9407060FE00CC000E8FAD5D1DC11F474
:10398000DCDE53DD0E94AB0514F4C6DC19F407E05D
:103990000093560152DD59F000915701013009F4AE
:1039A00072D71FD291D083D03CF700EFE6CF69DE0B
:1039B00076D0F1F701E8DCD564DE71D0F1F7BAD149
:1039C00000E00E940706B9DE0FE012C0A9DC91F406
:1039D000B4DE00915701013009F455D725DD0E946E
:1039E000AB0514F499DC31F4A8DE9ADCF1F707E0BA
:1039F0000093560122DD51F7D6D15ED031F49EDF1F
:103A00000E946D080E94780504C00E946D080E9403
:103A10007D050083118302E3009352010E947D081B
:103A2000ECDD87DE0E940E0404C0EAEAF2E00E94A8
:103A3000F8030091FA000730C0F30E94CF0474DC51
:103A4000F1F37BDE00915701013009F41CD7EDDC66
:103A5000C8D10E948025D8DD71F40E947F050081C5
:103A60001181012B09F462DF0E947A050081118126
:103A7000012B09F432D0009156010E3011F4B8D563
:103A800003C00FE00093560104D064F60E94750550
:103A90000895A7E2B1E0ED91FC9131970895EDE230
:103AA000F1E000811181003D27E0120708950450E4
:103AB00010402017310708950AE85AD502E0FBD1DB
:103AC0000091F40001300895E4E4F1E020813181B7
:103AD0000C94910506E000932C0100E0E7E2F1E090
:103AE0000083018308950E94B105CBDDE5DFD1F4A9
:103AF00025DF0E9464080E94780578DD54DCB0F16F
:103B0000A7DD39F40E94A20A0E94780582D075DDF3
:103B10007BD09ADD59F543DC49F50E944F080E949D
:103B2000780518C00E9464080E947D055FDD3BDCBB
:103B3000E8F08EDD39F40E94A20A0E947D0569D06A
:103B40005CDD62D081DD91F42ADC81F40E944F08B3
:103B50000E947D050083118304E3009352010E94BB
:103B600059084BDD0091F30000935C011CD1E1DDAD
:103B70000E940E0419C0E5ECF2E00E949C07E4DC10
:103B800016DC80F065DD29F4E7E8F3E00E94AB097C
:103B9000DBDC5ADD39F403DC29F4EEE8F3E00E94C3
:103BA000AB09D2DC0E9404040091FA00073018F33C
:103BB0000E94CF04B9DBF1F3C0DD00915701013061
:103BC00009F461D632DC0DD1ADD71EDD71F40E944F
:103BD0007F0500811181012B09F4A8DE0E947A057E
:103BE00000811181012B09F478DF009156010E301C
:103BF00011F4FED403C00FE0009356014ADF0CF02D
:103C0000B7CF0E94750508950091EE0000935C0106
:103C100008950083118303E300935201EAEEF0E07C
:103C200008950E94B1059A938A930BEF0E947C0736
:103C3000902F80E00CEF0E947C0710E00F5F1F4F79
:103C4000800F911F2BEF33E08C01012F0E94E706BC
:103C50002CEF33E0082F0E94E7060091DE0000936E
:103C6000F8000091DE00002319F401E00093DE006B
:103C70000091DE0000587CD40091F8000093DE0033
:103C8000C3DC31F45BDE0E9461080E94780504C049
:103C90000E9461080E947D050083118306E3009362
:103CA00052012091DE0030E004E1039F029FE0E03A
:103CB000F1E00082118239DE3093260104E60093A0
:103CC000FC00DFDCECDEF1F735D037DD0E940E04BE
:103CD00004C0EAEEF2E00E94F8030091FA00073017
:103CE000C0F30E94CF0420DBF1F327DD00915701E0
:103CF000013009F4C8D599DB74D086DC71F40E94D8
:103D00007F0500811181012B09F410DE0E947A05E4
:103D100000811181012B09F4E0DE009156010E3083
:103D200011F466D403C00FE000935601B2DE74F6BE
:103D300050DC089534D000E91CD0B1DEF1F70E94C8
:103D4000030310C003E01CD061F4F7DC00915701BD
:103D5000013009F498D50E94710619F405E00E941B
:103D6000070605D0D2DA00FFEDCF10D0089500E8A5
:103D7000FFC3FED34FEF20EA3FE000EA1FE0E3C3BA
:103D80000E940706009126010130089509B70F7BB4
:103D900009BF0E9403030FE000935601089500E05D
:103DA000009350010895FBDF00EAE3DF78DEF1F7CE
:103DB000DEDF0E94030310C004E0E2DF61F4BDDC3B
:103DC00000915701013009F45ED50E94710619F483
:103DD00005E00E940706CBDF98DA00FDEDCFD6DFC5
:103DE00008957B2F2A2E682F80E02AC0369A349BB4
:103DF000FECF24B115B100E0020F53D00E9491080C
:103E00000E946A080E9404040091FA00083070F3CE
:103E100002E0809F42D00E94AB0A43D0008311830E
:103E20003BD0A081B18138D0008111814DE20E9448
:103E3000E406A01BB10B1E972FD0A083B1838395FE
:103E4000843050F4082F0C5F07B900E02AD00083BB
:103E500001830093FA00D8CFE4E3F1E002811381FB
:103E600058DA02831383E4E3F1E00081118151DA2F
:103E700004831583E4E3F1E0048115814ADA0083C9
:103E80001183008111810539AEDB14F0969A0FD0B1
:103E9000862FA22DB72F0895829FF001EC5CFE4F74
:103EA000089522E0829FF001EC5CFE4F089500E04F
:103EB0000093250108958A93802F09B30C700C306C
:103EC00009F46CC009B302FB16F401E001C000E084
:103ED00007B900E0EDE4F1E0008301830EC0369AFB
:103EE000349BFECF44B135B120E0240F0E94A80AD4
:103EF000420F531F408351830395083080F30E9483
:103F0000AB0A00831183008111810A5A10400AF420
:103F100020DD212F220F220B322F0E94C3260E9468
:103F2000E02840E050E068EC71E40E947B270E94AA
:103F3000CE26EDE4F1E000831183813041F40E944C
:103F4000B20401E00093FB000E949F0502DC009197
:103F5000F700013019F5823009F522D024F00E94D3
:103F600052085CDBDCF40E9403030E940A0418D0B0
:103F70002CF421E10BEF14E00E942C030E945D075A
:103F80000E9452084BDB2CF421E10CE015E00E946A
:103F90002C0315DA99DAF1F70E9403038991089549
:103FA000EDE4F1E020813181EBE4F1E00081118169
:103FB0000E5110402017310708950E940E040AC0C8
:103FC0000091FA0010E0F801EA5EFE4F0E94B6048C
:103FD0000E9404040091FA00073090F308950E94B3
:103FE0000E0409C00091FA0010E0F8010BDA0E94FB
:103FF000B6040E9404040091FA000A3098F3089570
:104000000E940E0408C00091FA0010E08CDA0E94B1
:10401000B6040E9404040091FA000A30A0F3089547
:1040200019B31C701C3071F01091F700113051F46D
:1040300010915201163331F010915201112311F0F9
:10404000D89801C0D89A025019F00A9561F00895E5
:104050005F9B07C20CB1033709F003C25D9BFECF23
:1040600005E60CB908955F9BFCC10CB10337D1F58F
:104070005D9BFECF009152010CB90E940E0417C047
:104080005D9BFECF0091FA0012E0F4D100810CB9E3
:104090005D9BFECF0091FA00EDD111810091FA00F5
:1040A0000295007F000F010F0CB90E9404040091DB
:1040B000FA00083028F35D9BFECFA6DA19F40E94BF
:1040C0007A0502C00E947F0500810CB95D9BFECF7E
:1040D0009BDA19F40E947A0502C00E947F051181C3
:1040E0001CB90895003709F0CBC05D9BFECFBAD153
:1040F0005F9BFECF0CB1083231F4009152010023D6
:1041000051F467DB08C01091BE001093FD000093CE
:10411000BE005FDBAAD15D9BFECF0091BE000CB953
:104120005F9BFECF0CB1013011F401E001C000E053
:10413000009353010E940E0408C05D9BFECF0E94B5
:10414000BB0A00810CB90E9404040091FA000A30F5
:10415000A0F30E940E0408C05D9BFECF0E94B40A2B
:1041600000810CB90E9404040091FA000A30A0F307
:104170005D9BFECF0E947D0811811CB95D9BFECF27
:1041800000810CB95D9BFECF0E946D0811811CB9A6
:104190005D9BFECF00810CB95D9BFECF0E9467083E
:1041A00011811CB95D9BFECF00810CB95D9BFECFD8
:1041B0000E94640811811CB95D9BFECF00810CB97F
:1041C0005D9BFECF0E94610811811CB95D9BFECFF3
:1041D00000810CB95D9BFECF0091DE000CB95D9BA8
:1041E000FECF0091DB000CB95D9BFECF0091F40087
:1041F0000CB95D9BFECF0E945E0811811CB95D9BCE
:10420000FECF00810CB95D9BFECF0E94A20A1181F6
:104210001CB95D9BFECF00810CB95D9BFECF009168
:10422000EE000CB95D9BFECF0091BB000CB95D9B0D
:10423000FECF0E94590811811CB95D9BFECF008101
:104240000CB95D9BFECF0E944F0811811CB95D9B8C
:10425000FECF00810CB95D9BFECF0091F3000CB93D
:104260005D9BFECFFFD000915201002329F4BADA02
:104270000091FE000093BC0001E0009351010895FD
:10428000003509F0EEC00091BE000093FD005D9B7B
:10429000FECFE8D05F9BFECF0CB10093BE005F9BCA
:1042A000FECF0CB1009354010E940E0407C05F9B27
:1042B000FECF2CB10E94BB0A0E9403040091FA00B9
:1042C0000A30A8F30E940E0407C05F9BFECF2CB1FA
:1042D0000E94B40A0E9403040091FA000A30A8F375
:1042E0005F9BFECF0CB110E00E947D08008311831C
:1042F0005F9BFECFC4D05F9BFECF0CB10E946D08C8
:10430000008311835F9BFECFBAD05F9BFECF0CB1C1
:104310000E946708008311835F9BFECFB0D05F9B34
:10432000FECF0CB10E946408008311835F9BFECF17
:10433000A6D05F9BFECF0CB10E9461080083118361
:104340005F9BFECF9CD05F9BFECF0CB10093DE0045
:104350005F9BFECF0CB10093DB005F9BFECF0CB1E7
:104360000093F4005F9BFECF0CB10E945E080083B7
:1043700011835F9BFECF83D05F9BFECF0CB10E9469
:10438000A20A008311835F9BFECF79D05F9BFECF93
:104390000CB10093EE005F9BFECF0CB10093BB000D
:1043A0005F9BFECF0CB10E945908008311835F9B75
:1043B000FECF65D05F9BFECF0CB10E944F080083FB
:1043C00011835F9BFECF5BD05F9BFECF0CB1009350
:1043D000F3005D9BFECF46D005E00E94B50906E0E4
:1043E0000E94B50907E00E94B50909E00E94B509DD
:1043F00008E00E94B5090AE00E94B5090BE00E949E
:10440000B5090CE00E94B5090DE10E94B5090EE165
:104410000E94B5090FE10E94B5096FD977D802E271
:104420000E94B50900915401013099F40E944F098E
:1044300020F06FD810F401E009C06BD830F0009183
:10444000BE000E3110F402E001C000E00093F9005C
:1044500029D800915401002309F407D001E000930A
:104460005101089509E70CB908950091FD000093EA
:10447000BE000895019FF001EC5CFE4F089520817D
:104480000CB1008321830895FA93EA9320D04FB7AB
:104490001FB74BDA01E0009326010E947F052081BF
:1044A0003181232B21F00E949A050E946A08EBE2D9
:1044B000F1E00E9470071FBF4FBF03D0E991F9914F
:1044C00018950991199129913991499108954A9323
:1044D0003A932A931A930A930895FA93EA935A9374
:1044E000F6DF3FB72FB705E004BDEFE2F1E022D0E1
:1044F00044F0C49902C0C49A01C0C4980E946C1AC6
:104500000AC0E1E3F1E016D0B4F71BD9E3E3F1E030
:1045100000810A95008300913301002321F409B73B
:104520000F7B09BFC49A2FBF3FBFCBDF5991E991E1
:10453000F991189500811181EDE2F1E040815181FE
:10454000041715070895EFE2F1E000831183020FCD
:10455000131FE1E3F1E0008311834093330100E096
:10456000EDE2F1E00083018309B7006409BF08951B
:104570000FB9779BFECF0FB100934F0108952A9397
:104580001A930A932FB71FB706B30F700093560103
:104590001FBF2FBF09911991299118952093FA00F7
:1045A00002300091FA0012E041F4019FF001EC5B4F
:1045B000FE4F11D0EC5BFE4F04C05CDF0CD0EC5C16
:1045C000FE4F0E94A80A0417150714F42F5F3F4FEF
:1045D0000E94111A0895208131813595279589010E
:1045E000000F111F4091FA0052E0459FF00108951D
:1045F0008A9380E00E9403038093FA000091FA00FE
:10460000073098F4E6E5F2E00091FA0010E0E00FE0
:10461000F81F0E94FD03F2CF0E941F040E9489042C
:1046200023E007EB10E00E941C030E94211A09F40A
:1046300086C00E941D1A09F482C00E949019F9F4E4
:104640007CD800915701013009F41DD10E94141A41
:1046500000915201013309F4C5D100915201023396
:1046600009F44ED200915201033341F000915201FE
:10467000043321F000915201053309F453D2009123
:1046800056010E3091F60FE0009356018823E9F4AD
:1046900081E00E940E0408C0E1E7F2E00E94AB094D
:1046A0000E94911A0E9403040091FA000A3008F057
:1046B000B3CFEDE5F2E00E949C070E94D2060E9473
:1046C000960551F7E7E6F2E0E9CF8130B9F482E0F0
:1046D0000E940E040091FA000A3008F09DCFEBE72B
:1046E000F2E00E949C070E94D206EDE5F2E00E94F3
:1046F000AB090E94911A0E940304ECCF80E08093E2
:10470000FA0012C0E1E7F2E00091FA0010E056D0A2
:104710000E94021A2083EBE7F2E00091FA004ED0EB
:10472000E45FFE4F0E9403040091FA000A3008F093
:1047300073CF0E94960531F7E7E6F2E0E5CF0E94DD
:10474000211A21F40FE00093560141D00E941D1A56
:1047500019F50FE000935601882381F40E94960515
:1047600019F40E947F0502C00E947A050081118120
:104770000B5F1F4F008311832AD00EC0813011F4CC
:10478000A9D90AC007E000935601A4D941E020EA64
:104790003FE000EA1FE0D7DE0E947F050081118123
:1047A000083E23E0120734F007E0009356010E9410
:1047B000A11BCBD80E94030389910895E00FF81F35
:1047C00024910091FA00F801089500934A0100E055
:1047D00000932C0108958A9380E0009156010E30D9
:1047E00089F40E94D61B0E94A91B0E94461A29F434
:1047F0000091BC000093240105C0E4E2F1E00081D7
:104800000A950083009156010B3071F40E94D61B6B
:104810000E94A91B0E944A1A19F40E94C21B04C0DC
:10482000E4E2F1E00E947007DCDA0E94891900815D
:10483000118108370E94211B8CF096980E948519DF
:1048400000FF02C001E801C00AE819D00023A1F46A
:104850000E94CB0281E0809325010EC0008111816E
:10486000053612074CF4969A01E809D0013021F47C
:104870000E94CB0281E01BDB082F8991089578DE2E
:104880000091250108950E94B10563D820E030E031
:1048900001B944EC46BF04C00F5F1F4F2F4F3F4F7D
:1048A00046B7542F57FD02C088D0B0F386D078F4B5
:1048B00001B1087F003629F000EE18EC20E130E06D
:1048C00004C047D820E030E041E040935701012B7D
:1048D000022B032B09F05FC069D07CD017FFFDCFFE
:1048E00068D009F05ED079D0008711875FD072D090
:1048F00017FFFDCF5ED009F054D067D020853185F9
:104900004DD02087318752D065D017FFFDCF51D0D1
:1049100009F047D062D00287138748D05BD017FFD9
:10492000FDCF47D009F03DD050D02285338536D019
:10493000228733873BD04ED017FFFDCF3AD009F006
:1049400030D04BD00487158731D044D017FFFDCF2E
:1049500030D009F026D039D0248535851FD0248762
:10496000358724D037D017FFFDCF23D009F019D0D9
:1049700034D00687178704E806BF2CD017FFFDCF79
:1049800001B1087F083809F00CD01FD02685378583
:1049900005D0268737870E9475050895200F311F9F
:1049A0000895A8E5B1E0ED91FC91099404EC06BFEF
:1049B000089501B1087F00380895013442E41407D6
:1049C0004FE0240740E03407089503B110E0E4E32A
:1049D000F1E0089506B7102F089513B100E0E4E365
:1049E000F1E0089571D80E9474088CF40E94851932
:1049F00000FF0DC069D808525BD80CF4D4D9E7DEAB
:104A0000009326010E94921C0083018308950E9456
:104A10008D0500514DD81CF40CECD7DE10C00E945F
:104A20008D05015045D814F404EC07C00E94891983
:104A3000048115810E940C1B00EC00934A010E9426
:104A4000891957D00E949105005132D834F44ED0C4
:104A500000810D5F0083BBDE0BC00E94891949D025
:104A60000E949105015024D81CF440D00E94700788
:104A70002BD80A501DD82CF439D00081005D00835A
:104A80002FC022D80E94630724F430D00081005F39
:104A9000F6CF0E94081B4CF429D00081005F0083F0
:104AA000ECE2F1E00E9470071CC0008111810C5FF4
:104AB0001F4F0E9489190E940E1B14F01DD0F0CFC9
:104AC00005D80E9474085CF00E94AC1C0E948519F5
:104AD00000FF30D900E879DE0093260102C00CD037
:104AE00076DE01D0089500914A0142CDEAE4F1E07A
:104AF000089522813381089500E800934A010895C2
:104B00000E94641D06500E94581D14F40FEF06C049
:104B10000E94081B14F405ED01C000E800934A014F
:104B2000E2DF08950E948D050E94571D1CF453D0AA
:104B300000540BC00E948D050E9463072CF447D0DF
:104B400019F049D0045401C000EC00934A010E94BE
:104B50008919CFDF0E9491050E94571D1CF4009116
:104B60005C010DC00E948919C4DF0E9491050E945A
:104B700063074CF42CD039F000915C010A95B6DF44
:104B80001081100F10830E94641D0E94571D4CF469
:104B900000915C010295007FA9DF1081100F108346
:104BA00014C00E94641D0E9463075CF410D029F4B5
:104BB0009DDF0081005D008308C000915C010A95C3
:104BC000E9CF0E94081BA4F397DF8DDF08950091C1
:104BD0005C010023089500915C01000F000F08950F
:104BE0000FE90DBF00E00EBFC0E8D0E00E94B6287C
:104BF000002311F00E94C6280E94AB030E945B298B
:104C00000C945B291B2E0A2EDA0140E050E060E094
:104C100070E00E946C2839F400E010E04D934C9352
:104C200020E030E00CC0B901660F771F7E57572F88
:104C3000550F550B7D935C932F7730783F63A02DF4
:104C4000B12D08950024E8E0EA9532F0001F001C21
:104C50000416D0F3041AF8CF001F402D00950895D4
:104C6000FF27442312F4F1604195002312F4F095DC
:104C700001950E942226F0FD0195F1FD41950895D0
:104C80004A951AF015950795FBCF08950024112435
:104C9000EFE0001F111F001C111C0416150610F078
:104CA000041A150AEA95AAF7001F111FA001009522
:104CB000109508955195419550400895FF2755232B
:104CC00012F4F160F7DF112312F4F09507D00E947F
:104CD0004626F0FD03D0F1FDEDCF08951195019525
:104CE000104008954A952AF036952795179507950F
:104CF000F9CF089530952095109501951F4F2F4FAE
:104D00003F4F0895FF27112477FB660F771F089404
:104D100009F4771F679517F8EE27002437FB220F59
:104D2000331F089409F4331F279507F8089527FDCA
:104D30000EC0EE0F001F111F221F3A953230B8F738
:104D4000332319F427FD31E002C027FF30E0E038BB
:104D500021F400FF08940EF488940F4F1F4F2F4F3B
:104D60003F4F323038F4332319F427FD31E002C0CD
:104D700027FF30E03F3F31F0220F000C3795279599
:104D800008959DC0A2C0032E002012F40E947A262E
:104D9000E02F012F122F232F3EE9D0CFBDDF432F6D
:104DA0004F5758F0403258F000202AF00FEF1FEF15
:104DB0002FEF3FE7089530E884C0332782C0322FB9
:104DC000212F102F0E2F4F5141950E94722607FE62
:104DD00008950C947A26F901EE0FFF1F37FBFF3F71
:104DE00031F0EF2BE12BE02B8894B8940895E0305C
:104DF0001E070E0721F008949894B894089598948B
:104E0000889438940895FB01EE0FFF1F77FBFF3F56
:104E100031F0EF2BE52BE42B8894B8940895E03023
:104E20005E074E0761F3E7CFEEDF68F021F437232A
:104E3000262F8A010895372FFBCFE5DF20F00BF0F6
:104E400008957327EAF745C0C6DFE8F3B3F361F3CB
:104E5000DADFC8F383F3A1F355DF40175107620788
:104E6000730778F0332E372F732D322E262F632DB4
:104E7000312E152F532D302E042F432D302C012C85
:104E8000132C371739F0669557954795F795E040FD
:104E90007395F7CFE7FBEE0FE0E010245AF0EF0F29
:104EA000041F151F261F50F4279517950795E795A2
:104EB000339544CFEF0B040B150B260B3FCF302D52
:104EC000307822271127002708953FE7302920E86E
:104ED000F9CF302D3F672FEFF5CF95DFD0F3C9F332
:104EE000707837270895F5CF8EDF98F393F3F8CFD6
:104EF000307837279DCF6FDF60F37BF3A9F383DF33
:104F000040F3B3F3A9F3FEDE0124E8943F57E040F9
:104F1000370FEF1F12F0C9F603C03A3E80F26894D3
:104F2000E0E00A92AA933A93AA2733242224332753
:104F3000049FF001059FF00D712D731F149FF00D5C
:104F4000711D221C069F700D211C331C159F700DB6
:104F5000211C331E249F700D211C331E169F200C14
:104F6000311CAA1F259F200C311CA31F269F300C2B
:104F7000A11D39915EF43395A695379427947795C2
:104F8000F795E79533953130BCF316C0AA2322F08C
:104F9000332351F4339510C0339571F4A9910990DE
:104FA00094CFA7FD09C03A95EE0FFF1F771F221C73
:104FB000331CAA1F3230A8F7E894FE2B09F068943E
:104FC0002A2F8101E72FA9910990C1CE1CDF10F093
:104FD0000BF086CF7ECF17DFE9F3E0F3032E072631
:104FE0006ECF032E072671CFF6DEA0F37BF399F385
:104FF0000ADF80F39BF3A9F385DE012427FD06C0B9
:10500000000F111F221F3150E040F8CF67FD06C08E
:10501000440F551F661F7150F040F8CFE894371BBE
:10502000EF0B3158EF4F2AF0EE23E9F63F3FD9F26C
:1050300003C03A3EA8F26894E0E0F0E01124139433
:1050400040175107620740F03A953F3F09F46894D2
:10505000000F111F221FEE1F041B150B260BEF0B59
:10506000000F111F221FEE1F77E17A95A2F004179F
:1050700015072607EF0730F0041B150B260BEF0B67
:10508000089401C08894111C221C331C000F111FAE
:10509000221FEE1FEACF401751076207FE0718F0E4
:1050A00021F4E0E803C0EFEF01C0E0E0332311F0AA
:1050B00056F4E894369427941794E79508F4689486
:1050C00033953130BCF3012D122D232D40CE9BCED4
:1050D00098940895189408957EDED0F3C1F393DE7A
:1050E000B8F3041715072607370708958CDEA0F0DC
:1050F00072DE90F029F0E32FE7273AF47317089552
:1051000082DE51F04EF00894089504171507260723
:10511000370719F016F4B8F78894089574DEE0F3B1
:105120005ADED0F3E7DFC0F308940895BA92AA924A
:105130009A928A927A926A925A924A92BA93AA93CD
:105140009A938A930895BB84AA84998488847F80E3
:105150006E805D804C80BB81AA8199818881F0E05E
:105160000FB6F894CE0FDF1F0FBE089501E008952B
:1051700020E002D0E9F708952D9301501040202F30
:10518000212B08952591F8DFE9F708958CEB92E53E
:10519000FC0105911491FC013296A591B491FC019A
:1051A000349625913491422F432B19F0F901EADF0F
:1051B00001C0DEDF069612E5883C910748F30895AA
:1051C0000E94962822974801590141E050E060E092
:1051D00070E00E94762898F440E00E946C2829F440
:1051E00000E010E020E030E05DC001E2EFE5F1E03A
:1051F000008351830FEF1FEF2FE73FE753C0AE014E
:105200000E940226C801D90145EC53E062E47FE325
:105210000E9424274AE151E562E17FE347D0A801DB
:10522000B9018C019D010E94F427A201B3010E94E3
:1052300024272801088100FF16C00A9542E00E9439
:105240003026802F820143EF54E065EB7FE30E941C
:105250007B2737FB220F331F380F3695279537F9F9
:10526000C801D9010CC042E00E943026C201D90118
:10527000B7FBAA0FBB1FB00FB695A795B7F98C0166
:105280009D0140E050E060E87EE310D0840195018C
:10529000AC01BD010E94F427A801B901820193016C
:1052A0000E9424272296ECE00C94A3280E947B27DE
:1052B00028013901089500008895FECF1E00A00046
:1052C000C852A300BE00000020202020006C2F68E0
:1052D0000073006D00250043003D004C005200208B
:0652E00020200001020184
:00000001FF
